:1000000090C097C096C095C094C093C092C091C054
:1000100090C08FC08EC08DC08CC08BC08AC089C07C
:1000200088C000060C12181E242A30363C42484E66
:10003000545A60666C72787E848A90969CA2A8AEB0
:10004000B4BAC0C6CCD2D8DEE4EAF0F6FFFFFFFFB8
:10005000FFFFFFFFFFFFFFFFFFFFFFFFFFFFFFFFB0
:10006000FFFFFFFFFFFFFFFFFFFFFFFFFFFFFFFFA0
:10007000FFFFFFFFFFFFFFFFFFFFFFFFFFFFFFFF90
:10008000FFFFFFFFFFFFFFFFFFFFFFFFFFFFFFFF80
:10009000FFFFFFFFFFFFFFFFFFFFFFFFFFFFFFFF70
:1000A000FFFFFFF9F3EDE7E1DBD5CFC9C3BDB7B182
:1000B000ABA59F99938D87817B756F69635D575160
:1000C0004B453F39332D27211B150F090000000038
:1000D0000000000000000000000000000000000020
:1000E0000000000000000000000000000000000010
:1000F0000000000000000000000000000000000000
:1001000000000000000000000000000000000000EF
:1001100000000000000000000000000000000000DF
:10012000000011241FBECFE5D1E0DEBFCDBF1AD045
:10013000BBC066CF0F931F9300E010E09801061735
:1001400017072807390759F0E7E8F3E13197F1F786
:1001500000C000000F5F1F4F2F4F3F4FF0CF1F9188
:100160000F910895F89487E893E10197F1F700C0A3
:10017000000080EF809374008AB38F608ABB80E0B8
:1001800090E001968F3F910511F480E090E0682F98
:10019000582F5E6F20E8422F4523322F36952BB320
:1001A0002F602BBB442379F0232F000000000000B8
:1001B00000000000000000000000000000004BB341
:1001C000407F4BBB06C0000000002BB3207F2BBB41
:1001D000232F0000000000000000000000000000CD
:1001E0003111D9CF606C20E8422F4623322F36954B
:1001F0002BB32F602BBB442379F0232F000000008A
:1002000000000000000000000000000000000000EE
:100210004BB3407F4BBB06C0000000002BB3207FD8
:100220002BBB232F00000000000000000000000096
:1002300000003111D9CF20E8422F4523322F3695C7
:100240002BB32F602BBB442379F0232F0000000039
:10025000000000000000000000000000000000009E
:100260004BB3407F4BBB06C0000000002BB3207F88
:100270002BBB232F00000000000000000000000046
:1002800000003111D9CF2BB32F602BBBEFE4F3EC7F
:100290003197F1F700C000002BB3207F2BBBF2E4B5
:0C02A000FA95F1F700C06DCFF894FFCF85
:00000001FF
